:020000020000FC
:10000000B1CD00000000000020C0AFC194C00000CE
:1000100000009EC000000000000000000203040673
:10002000080C10182030406080000406080C1018DE
:100030002030406080A0C00000070F1F3F000D0D62
:1000400004050D050305030302004FB662FD0EC053
:10005000552009F00994C52DC095089483FDC795D6
:10006000C4BDC093A10064604FBE1895C0916400E8
:10007000089483FDC795C4BDC093A1006B7FC09158
:100080006400CF3F09F420C070FF02C082FD05C0AC
:100090004FBEC19897989598189575FD0EC065FD4F
:1000A0000CC0C091B300C0FD9298C1FD9398C2FDF1
:1000B0009498CAEFC095CA95F1F7C198979895980A
:1000C0002092A1004FBE189524BCCC27C064C8BFA5
:1000D0006460F6CFC0CF70FFBECF65FDBCCFC19AC4
:1000E000BACF70FFB8CF65FDB6CF979AB4CF70FF87
:1000F000B2CF65FDB0CF959AAECF929A70FFABCFDD
:1001000065FDA9CFC7E0CA95F1F7C19AA4CF939A2C
:1001100070FFA1CF65FD9FCFC7E0CA95F1F7979A11
:100120009ACF949A70FF97CF65FD95CFC7E0CA9597
:10013000F1F7959A90CF4FB6C9B7CF7EC9BF6E7F02
:10014000CCB5CE0DDDB5DF1DDBBDCABD4FBE1895EC
:100150003FB68F7EA9B7A072A2118061A9B7AF7D0B
:10016000A9BFA9B7AE7FA9BF7894A0916800AA23C0
:1001700041F085FD2BC0A0916800AA95A09368006E
:1001800025C040E050E085FD15C0A6B396FDA095C2
:10019000A0FD4FEFAEB5A06496FDAF7BAEBDAA2724
:1001A000A062A8BF8D7FA6B396FDA095A0FD5FEFCE
:1001B000451739F7A8E161FDA093680085FD03C0EC
:1001C000A8E1A093680040939700816085FD0EC070
:1001D000A0916900AA2331F0A0916900AA95A0938B
:1001E000690004C08061AA27A062A8BF80FF37C051
:1001F000A09197004A2F61FF8E7F85FD1CC0A091C2
:10020000B600A430C1F4403F08F040EFA42FA295FF
:10021000AF704A0F5091B800533069F0A695A6957B
:1002200050FD01C0A69552FD03C0A41B4A2F03C078
:100230004A0F08F44FEF40936100A72FA67079F0A2
:10024000A0916D00A695A69556E0A50F509161006E
:10025000A50FA093610018F4AFEFA0936100409147
:10026000B600443009F03EC0A0916100A093630045
:1002700040916300A0919C004A1708F04A2FA0917A
:100280009E004A1708F04A2F542EA091A200AA23DC
:1002900009F422C0542F5A1B10F4A42F50E0BA2E98
:1002A0008894AA1FAA2EA091A400A095AA22A50E08
:1002B00058F0A091A300A21509F0AA95AA0EA09348
:1002C000A30048F04A2D08C0A091A300BA1608F078
:1002D000A395A093A3004FEF409364007F7D485FF8
:1002E00008F07062A52DA03408F06860A09160004D
:1002F000A395A093600059F0F894A9B7A160A9BF95
:1003000084FF03C0A9B7A062A9BF3FBE1895A09102
:100310007400A395A093740041E0509168005523A8
:1003200029F085FF03C05A9550936800A09197006B
:10033000A13018F020929A000DC020929B002092CC
:10034000A500A0919A00AF5FA0939A0018F0AFEFBC
:10035000A0939A00F894A9B7A160A9BF84FF03C035
:10036000A9B7A062A9BF3FBE18953FB646B557B51D
:100370008F7EA9B7A072A2118061A9B7AF7DA9BF76
:10038000A9B7AE7FA9BF789481FD25C0AEB5AF7B7C
:1003900096FDA064AEBD8260A6B396FDA095A0FFB9
:1003A00005C0409365005093660041C1AEB5A0649E
:1003B00096FDAF7BAEBDAA27A062A8BF8D7F85FF4B
:1003C00001C028C140E0A6B396FDA095A0FD22C1C2
:1003D0004093970011C1AEB5A06496FDAF7BAEBD52
:1003E0008D7F61FF72C0AEB5AF7B96FDA064AEBDE0
:1003F000AA27A062A8BF8260409392005093930006
:10040000A09090004A19B09091005B09BB24A22CE7
:100410004C38520518F42092960049C0A091D6009D
:10042000AA2359F1483C520528F4A0E1BA2EAAE0CB
:10043000AA2E23C04836A1E05A0728F4A8E0BA2E15
:10044000AFE0AA2E1AC0403DA2E05A0728F4A4E06B
:10045000BA2EAEE1AA2E11C0403AA5E05A0728F400
:10046000A2E0BA2EACE3AA2E08C04839A8E05A0789
:1004700020F4A1E0BA2EA8E7AA2EC42EA0919400E1
:10048000CA1AD52EA0919500DA0ADD202AF4AFEF22
:10049000C094D094CA1ADA0A20929600A8E0A2105A
:1004A000A0E0CA14DA0618F4A1E0A09396004093E5
:1004B0009400509395004091920050919300409386
:1004C00090005093910002E097C0A09165004A1BF4
:1004D000A09166005A0B94FD82C093FD80C092FDEE
:1004E0007CC086FF03C0D52EC42E0CC05695479500
:1004F00091FD73C05695479590FD6FC0D52EC42EC3
:10050000D694C79461FD19C0AC2DAC51AD2DA2405D
:1005100008F005C0DD2089F4AC2DA85C70F4A09132
:100520006700A395AA2311F0A0936700AA3008F4EE
:1005300071C02092970081606DC0A0916700AA23CE
:1005400019F0AA95A0936700A22C5091BC0097FDCA
:1005500006C0A090CA00533011F4A090D200AAEFB8
:10056000AA0EA22DA21DCA18DA0A4FB74170533045
:1005700049F4442321F087FD05C0806803C087FF4C
:1005800001C08F77442359F0533031F4AFEFC0945A
:10059000D094CA1ADA0A03C040E050E020C05330B9
:1005A00049F4CC0CDD1CAAE0CA1AD20818F4A0E069
:1005B000CA2ED22CAFEFCA16D20418F04FEF50E07B
:1005C0000EC0A091AE00CA9E412D000C441F50E009
:1005D00008F012C04FEF50E00FC05695479594FFBA
:1005E00007C0552309F04FEFA42FA6954A0F521DBF
:1005F0004F3F520508F04FEF40939700816061FF35
:1006000009C0AFE1A095A923AB299A2F8F7DBB200C
:1006100009F48062A8E1A093680085FF03C0AAE006
:10062000A093680061FD03C085FD01C08F7E85FD3C
:1006300003C0A6E0A0936900F894A9B7A160A9BF80
:1006400084FF03C0A9B7A062A9BF3FBE189511E0FF
:100650000AC013E008C01AE006C01EE104C014E698
:1006600002C018EC00C005E1BB27BA95F1F70A9566
:10067000D9F71A95C1F708952AE338E709C020E3AE
:100680003CE806C02AE234EB03C025E238EC00C0A7
:1006900012E095FD9F7D95FF9062BB27939ABA95D6
:1006A000F1F7979ABA95F1F79798BA95F1F7939869
:1006B000BA95F1F7C19AB091AF00BA95F1F7C19828
:1006C000B7E8BA95F1F71A9521F7022FB22FBA952C
:1006D000F1F70A95D9F73A95D9F6939A0895221B1E
:1006E00039E0001F3A9509F40895221F211B18F4E0
:1006F000210F8894F6CF0894F4CF622C722CB0E0CE
:100700008894B395221F331FE0F737952795889477
:10071000912E802E020B130B10F4192D082D10F4BE
:10072000889401C00894661C771CBA9571F7172D40
:10073000062D0895322D11232AF43A95009510952F
:10074000031B130BF894029F712C002D129F912C08
:10075000802C7894780C172D921C292DB4E06B2EE8
:100760002695179507956A94D9F7332321F00095BC
:100770001095031B130B08950091B6000430A1F1EE
:10078000B0919700B15008F010C0B0916100B093E3
:10079000630020927F0020928000209281002092AE
:1007A0008200209283006F7B1FC06090B60060645F
:1007B000B0916100B093620008E317EC20917A00D9
:1007C00030917B0036952795B62DBA9541F0369538
:1007D0002795B62DBA95BA9511F0369527958DDFE8
:1007E00000937F0010938000089500917F00B091E6
:1007F00062000B1B10918000120928F40038BFEF33
:100800001B0740F009C00F37120508F405C00FE7B9
:1008100010E002C000E81FEF0093840010938500F1
:10082000089500918400B09181000B0F1091850014
:10083000B09182001B1F20E03091850033230AF421
:100840002A95B09183002B1F1AF4203F40F00AC074
:100850002F3008F407C00FEF1FEF2FE003C000E0B8
:1008600010E020EF30916300B0919C003B1718F42A
:10087000323030F009C0B0918500BB235AF004C07B
:10088000B0918500BB2332F4009381001093820065
:100890002093830008952091D80000918400000FD8
:1008A00010918500111F46DF11232AF40038BFEF95
:1008B0001B0740F009C00F37120508F405C00FE709
:1008C00010E002C000E81FEF002352F0B091620078
:1008D000B01B0B2F18F0013008F00AC001E008C06F
:1008E00000950F5FB09162000B0F08F001C00FEF91
:1008F0000093860008952091D90000918200109104
:10090000830018DF11232AF40130BFEF1B0740F0EA
:1009100009C00F3F120508F405C00FEF10E002C038
:1009200001E01FEF112352F0B0918600B01B0B2F96
:1009300018F0013008F00AC001E008C000950F5F10
:10094000B09186000B0F08F001C00FEF0093630019
:1009500008950FEF677F71FD29C072FD09C06860BF
:10096000B0917B00BA3020F0B52DB03408F4677F29
:10097000B091D500BB23D1F0B0917B00BB23B1F087
:100980000FEF10917B00ABDEF894B091730072FD15
:10099000B5E00B9F112D002D7894112309F00FEF76
:1009A000B0919F000B1710F400919F0000939E00E0
:1009B000089500917A0010917B0000541140B0918D
:1009C0009E0010F4BA9501C0B39511F0B0939E004B
:1009D000089500C008952091B700B6B1B6FDFBCFD1
:1009E00004B115B1B6B1BF77B6B9B091AC00B3954B
:1009F000B093AC00B83060F12092AC00B091D4005C
:100A0000BB2321F1112329F0B091AD00BF3F61F06C
:100A100009C0B091AD000B1739F020F4BB2321F0D1
:100A2000BA9502C0B395E1F300919C00B093AD007C
:100A3000BA3F50F400ECB93F38F400E8B83F20F476
:100A400000E4B73F08F400E000939C00777F08952E
:100A500010919C00B0E11B0F08F41FEF10939C0055
:100A6000B091B600B43081F000919C00B091630069
:100A7000B01B10F400916300B0919E000B1708F0BA
:100A80000B2F502E00936400B091AC00B73009F4E6
:100A90007860089502E3F894B091DA000B9F012D7D
:100AA000000C001F7894B0919C000B1710F000917F
:100AB0009C000093610000936300502E009364003B
:100AC00000939F00089520927A00B0EFB0937B00CE
:100AD0000895F8940CB51DB5209174007894309168
:100AE0007500609076000093750010937600031BEC
:100AF000160971FD03C076FD81C02BC07090770090
:100B0000209377002709222311F00FEF1FEF809029
:100B1000780090907900309378006092790069189D
:100B2000161910937C000091750010917600081939
:100B3000190920917A0030917B0036952795020F94
:100B4000131F10F40FEF1FEF00937A0010937B0038
:100B500029C020917A0030917B003901B4E08B2EBE
:100B6000B2E09B2E343010F08A949A94383010F012
:100B70008A949A94769467948A94E1F726193709AF
:100B8000992021F0169507959A94E1F7200F311FCF
:100B900020937A0030937B0028F43FEF30937A0063
:100BA00030937B00323008F4706471FF02C0B3E010
:100BB0000DC0B091C60000917100023838F0B395B5
:100BC000003A08F0B395B63008F0B5E09B2EB4E0DB
:100BD0008B2E10917B0000917A0024E016950795EA
:100BE0002A95E1F70819120928F0B02FB250B12F59
:100BF000B20910F402E010E0980126C020917A00BA
:100C000030917B003901769467946694669466947B
:100C10002619320906950695200F321D20937A0079
:100C200030937B00323008F07F7B04E036952795C7
:100C30003695279526952695201B10F0223008F42E
:100C400022E089019090C60060FDFECFE0908C000C
:100C5000F0908D006160B9B7B061B9BF380176FD21
:100C600044C07694679400938C0010938D00B92D46
:100C7000B330E1F0B0FD04C0060D171D930106C0AE
:100C8000000F111F0250120922E030E0B92DB330DD
:100C900068F020938E0030938F00009388001093AB
:100CA000890060928A0070928B003DC000938E0094
:100CB00010938F00209388003093890060928A00FF
:100CC00070928B0071FF10C0B0916D00B33060F076
:100CD00000918F0010917C001595010F28F022F0F3
:100CE00020928E0000938F001EC0669400938C00AB
:100CF000B92DB33091F0B0FD03C0060D262D03C011
:100D0000000F025022E0B92DB33038F020938E004E
:100D10000093880060928A0006C000938E002093A2
:100D2000880060928A0000917D0002FD035001302E
:100D300029F495FD0AC0B0E0B7B909C0023019F432
:100D4000B7E0B7B904C095FDF6CFB6E0B7B90091EA
:100D5000A400000F10F4BBE60B270093A40060FD75
:100D6000FECFB2E0B0936E006160B9B7B061B9BFB9
:100D7000B72FB670A1F020917A0030917B003695A4
:100D80002795F8940CB51DB5020F131F1BBD0ABDA6
:100D90006160B0E1B8BFB9B7B061B9BF78940895E8
:100DA000606120927E0020E067FD20E206C0606165
:100DB00020927E0020E267FD20E0789401E076FD3D
:100DC00011C0B72FB67009F06F7EB0917B00B5509F
:100DD00048F002E0B55020F003E0B55008F006E01E
:100DE00071FD0AE060FD12C0B0917E00BB2371F07E
:100DF00071FF08C0B0916D00B33020F0B0916E006B
:100E0000BA9519F4789470615CC0AEDF78940000F4
:100E10000000F89476FD16C010917B00173008F0A2
:100E200017E0B5E01B0F72FD10E183FF110F62FFA9
:100E3000110F71FD12E8B4B56090A100B61990F2DF
:100E4000B10B80F2B0B7B77FB0BFB8B1B0B7B86080
:100E5000B0BFB0917E00B395B0937E00B8B176FD7F
:100E600006C0B1E071FDB2E0BA95F1F7B8B1B07269
:100E7000B21709F01BC071FF05C003950A3008F0D6
:100E80000395B0CF64FF99CF6F7E3CB56DB4709081
:100E90007A0080907B00370D681C6BBC3ABD6160A6
:100EA000B0E1B8BFB9B7B061B9BF87CFB0916D003D
:100EB000B23008F482CF64FD80CF0A9509F092CF5A
:100EC0007F7E20918E0030918F00F894B0E1B8BF02
:100ED0000CB51DB5020F131F1BBD0ABDE0908800A5
:100EE000F09089006160B9B7B061B9BF7894B72F4D
:100EF000B67039F0B0916D0072FFB395B0936D008C
:100F000009C074FF07C067FD05C064FD03C0BF9141
:100F1000BF91E0C4089500E063FF03C064FF01C017
:100F200001E0F89410917100B7E01B9F212D102D66
:100F30007894200F26951795269517952695179541
:100F400010937100183718F4B8E7B093710000914E
:100F50007100B09172000B1720F06062C1989798F1
:100F6000959860FDFECFE0908A00F0908B00616064
:100F7000B9B7B061B9BF0895B2E095FD07C0F89464
:100F8000B0937D00939A92987894E5C0F894B093CA
:100F90007D00939A94987894DEC0B3E082FF24C0D9
:100FA00095FD11C002E0F894B0937D00E7E8F0E011
:100FB0000093B3009598949A62FF02C0979A01C07B
:100FC00093987894C8C002E0F894B0937D00E7E865
:100FD000F0E00093B300C198929A62FF02C0979A22
:100FE00001C093987894B7C095FD0BC0F894B09366
:100FF0007D00E1E7F0E0959862FF01C0979A789450
:10100000AAC0F894B0937D00E1E7F0E0C19862FFD8
:1010100001C0979A78949FC0B4E095FD07C0F894FA
:10102000B0937D00929A9498789495C0F894B09378
:101030007D00949A929878948EC0B5E082FF24C087
:1010400095FD11C001E0F894B0937D00EDE7F0E06C
:101050000093B3009798939A62FF02C0C19A01C0AF
:101060009298789478C004E0F894B0937D00E1E918
:10107000F0E00093B3009798939A62FF02C0959AAC
:1010800001C09498789467C095FD0BC0F894B09314
:101090007D00EBE6F0E0979862FF01C0C19A78947A
:1010A0005AC0F894B0937D00E7E7F0E0979862FFAC
:1010B00001C0959A78944FC0B6E095FD07C0F894AA
:1010C000B0937D00949A9398789445C0F894B09327
:1010D0007D00929A939878943EC0B1E082FF24C03C
:1010E00095FD11C004E0F894B0937D00E1E9F0E0D3
:1010F0000093B300C198929A62FF02C0959A01C012
:101100009498789428C001E0F894B0937D00EDE7BE
:10111000F0E00093B3009598949A62FF02C0C19AE0
:1011200001C09298789417C095FD0BC0F894B093C5
:101130007D00E7E7F0E0C19862FF01C0959A7894DE
:101140000AC0F894B0937D00EBE6F0E0959862FF5A
:1011500001C0C19A78946F7D08952AE630E0F901C4
:101160002092B300C19897989598929A939A949ADE
:101170006B7F0895A4EBB0E009E00D9309E00D93B7
:1011800004E00D930FEF0D9303E00D930FEF0D931C
:1011900009E00D9303E00D9301E00D9301E00D9341
:1011A000A0ECB0E001E00D930FEF0D930D930D93C4
:1011B0000D930D9303E00D930FEF0D930FEF0D9330
:1011C0000D9305E20D9300ED0D9308E20D9300E5FC
:1011D0000D9304E00D930FEF0D9302E00D9300E0EB
:1011E0000D930AE70D930FEF0D9300E00D9301E0CF
:1011F0000D9300E00D9303E00D9308952091BB0043
:101200008B7F233009F48460B091BC00B33019F0B7
:101210009F7DB1FD90629F7BB091BD00B1FD906458
:10122000223011F0886001C0877F08950A95E00F91
:10123000F21DB4910895ECE1F0E00091B400F6DF06
:10124000B093D800ECE1F0E00091B500EFDFB0938F
:10125000D900EAE2F0E00091BA00E8DFB093DA00EA
:10126000B091D0000FEF1CE0B23011F400EA1AE0A8
:10127000B33011F402E815E000937200109373008C
:10128000E8E3F0E00091D700D1DFB093A200089529
:1012900008952091CA003091CB00B091BC00B330CA
:1012A00009F43E5097FF02C020E03FEFB32FB21B7E
:1012B0006B2EB25810F4B2E86B2E00E00395609EDE
:1012C000B12DBD57D8F30093AE0008959068E1DFCB
:1012D000C4D920E030E0B0E16B2EBBD9B0919700CB
:1012E0002B0F321D6A94C9F7B4E036952795BA954D
:1012F000E1F7822E9F77CDDF0895F894E3E0F0E0E8
:10130000B9E0B7BFB491B078C1F3F894A895B1B57E
:10131000B861B1BDB0E0B1BDB4E0BEBFBFE5BDBF17
:101320001CDFB0E0B8BBB2E1B7BBB0E0B5BBB0E02A
:10133000B4BBBCE1B2BBBCEBB1BB2224A0E0B0E0CB
:101340002D92AA31E9F7A0E6B0E00FEF2D920A95B1
:10135000E9F7B1E0B093A4000DDFECD2B6B1B46010
:10136000B6B90091CC000093AF00B1E0B0936A0031
:10137000F89477D981D971D982D96FD983D96DD9A8
:10138000F8940AEF1AEFA6B396FDA095A0FF1FC030
:101390001A95C9F70A95B1F7E0E0FCE1B591B43EC2
:1013A00039F4B591B03E21F4B591BF3F09F40CC0BA
:1013B000E0E0F395F395B591B83F49F4B591B439B0
:1013C00031F4B591BA3A19F4EE27F695099416DF7F
:1013D00032DF5EDF5EDF0091CC000093AF00BDDE48
:1013E000B2E0B3BFB2E0BEBDB2E0B5BDB1E5B8BFDB
:1013F000B9BFB0B7B77FB0BFB8B1B0B7B860B0BF12
:1014000026D97894E6DABEB5B06496FDBF7BBEBD42
:10141000B9B7B062B9BFBB27B062B8BF8D7F21D961
:10142000626033E02CE0B0919600BB2321F42CE005
:101430003A9509F4A5CF11D980FFA2CF8E7FB09144
:101440009700B23078F3B92FBF71009199000093E3
:101450009800B0939900B01729F72A9521F76D7F6E
:10146000BEB5B06496FDBF7BBEBDBB27B062B8BF42
:101470008D7FB091D600BB2321F48062B92FB0706C
:101480009B2F8F7B20926700EAD885FF05C0B09123
:101490006700BA3008F08064DCD802E085FF01C044
:1014A00000E0B0919700B017B8F3F894E5D8E4D80D
:1014B000E3D87894D6D820928700B091BC00B3309E
:1014C00009F474C0C6D8B091C000B13008F46EC041
:1014D000B0916A00B13008F469C085FD18C0B091C0
:1014E0009700BF3F08F462C0F894CFD87894B7D87B
:1014F000B0919700B130C0F7F894BED8ACD8BCD842
:101500007894ADD8B0919700BF3FB0F3D4C2B3E0A8
:101510009B2E9068F894BDDE7894A1D8F8949F77BC
:10152000B8DE80909700B0919700BF37789408F4A8
:1015300045C08DD8F894A9D878949A9451F7C6DE0E
:10154000B82DB550B093CB008CD8F89420D286D269
:101550007894BAE09B2E9068F8949BDE78947FD8BC
:10156000F8949F7796DE80909700B0919700BF37F0
:10157000789478F76CD8F8947FD86DD87DD8789423
:101580009A9449F7A3DEB82DBB5FB093CA0069D81F
:10159000F894FDD172D2789462D8F8947ADE789477
:1015A000B0919700BF3F08F498CF85C20091970093
:1015B000B09187000B1710F00093870050D801E01E
:1015C000B091BC00B35009F405E0B0919700B0179A
:1015D00008F073CFF89459D858D857D8789441D890
:1015E00020926A0020926B0020926C00B0916B00F8
:1015F000B395B0936B00BF3F69F5B0916C00B395A4
:10160000B0936C00B091CE0009E1BA9559F002E3B5
:10161000BA9541F00DE7BA9529F00AEFBA9511F0A5
:1016200020926C00B0916C00B017A0F0B0916C00EB
:10163000BA95B0936C00B4EBB0936B00B091CD0051
:10164000B093AF00F89421D87894B091CC00B093C7
:10165000AF0005D800D8B0916800BB2319F485FF0E
:1016600001C08ECE01E085FD01C006E0B09197007B
:10167000B01708F4BBCFB091BC00B35009F0EFD75E
:10168000B0916800BB2309F47BCEF89466DD20920C
:1016900061002092620020926300522C209264002C
:1016A0002092A3007894B091B900BB0FB093A00032
:1016B00020927F0020928000209281002092820060
:1016C000209283002092AC0060E070E020927100D4
:1016D000B8E0B093AC007860BAD7B2E073FDB1E087
:1016E000B7B9B6B1B068B064B6B9B6B1B6FDFDCFA2
:1016F00004B115B1B6B1BF77B6B9112309F00FEF38
:101700000093AD0068D9B8E0B093AC0078608090E9
:10171000BB00B2E0B093BB0071DD8092BB00F894D7
:10172000BFEFB0939C00B6D9B0916100B0939C001C
:10173000B0939D00B0939E007894B1E0B0936100A7
:10174000B09363005B2EB0936400B093A600B09199
:101750009B00B093A500B091BC00B33019F49F7DFD
:1017600087FD90627160726020926D00A5DCB5DC2F
:10177000AAD9AFD9A8D9ADD9A6D906C0F8943EDD6B
:1017800078942092AC00777F12DBF6D7C4DBF4DBD1
:10179000A0D906DB66FD29D876FFDBD876FD09D90E
:1017A000BADBFBDB96D903DB66FD3BD8B4DB34DC6C
:1017B00090D9F6DA66FD6FD8AEDB3FDC8AD9F7DA6E
:1017C00066FD99D8A8DB78DC84D9EADAB2E073FD4B
:1017D000B1E0B7B9B6B1B068B064B6B99CDB7DDC36
:1017E00078D9F9D871FF26C067FD24C0B0919F0059
:1017F000B0939C00B0939D00B0919B00B093A50066
:10180000B1E0B093A60018E12CE0B0916D00B117E3
:1018100058F07D7F746020936F00B0919F00B0936B
:101820009C00B0939E0006C0B0919700B13008F0C4
:10183000ABCF5AC072FF10C067FD0EC0B0916F00F1
:10184000BA9511F47B7F9ACFB0936F00B091970057
:10185000B13008F099CF48C020927000B0919A0042
:101860000AEFB01708F040C085FF04C0B0916800CF
:10187000BB23D1F1B091BC00B33081F495FD03C01E
:1018800087FD04C00BC087FF01C008C067FD06C00C
:101890006068B0919F00B0939C008BCF00EF67FF12
:1018A00005C0B0919F00B0939C0000E2B0917B0016
:1018B000B01708F469CF67FF17C06F779F7D87FD6A
:1018C00090627460B2E1B0936F00B0919F00B093EA
:1018D0009C005ACFB0917000B395B0937000B09156
:1018E0009700BB2309F002C020927000F89435DC09
:1018F0008090BB00B2E0B093BB0080DC8092BB0064
:10190000209261002092620020926300522C20926B
:1019100064002092A0007E7F789499D61EDCB6B138
:10192000B460B6B985FF05C0B0917000B53008F05D
:1019300027CD58CEEDE0F0E023D0053509F01BC0EF
:10194000EEE0F0E01DD00A3A09F015C03AE0A4EB51
:10195000B0E0E3E0F0E014D00D9331963A95D9F77A
:1019600038E1A0ECB0E0EFE0F0E00AD00D93319662
:101970003A95D9F702C0FEDB0AD0E7E2F0E008951D
:10198000E199FECFEEBBFFBBE09A0DB308951ED0E8
:101990003AE0A4EBB0E0E3E0F0E00D910FD0319637
:1019A0003A95D9F738E1A0ECB0E0EFE0F0E00D9126
:1019B00005D031963A95D9F712D00895E199FECF26
:1019C0000DBBEEBBFFBBE29AE19A0895EDE0F0E0BB
:1019D0000FEFF4DFEEE0F0E00FEFF0DF0895EDE061
:1019E000F0E005E5EBDFEEE0F0E00AEAE7DF08957E
:1019F0003091B0000091B100313011F40093B40087
:101A0000323011F40093B500333011F40093B60076
:101A1000343011F40093B800353011F40093BA005B
:101A2000363011F40093C600373011F40093BB0038
:101A3000383011F40093D700393011F40093D000FE
:101A40003A3011F40093BC003B3011F40093BD0018
:101A5000089525E006D62A95E9F708950DD60FD604
:101A600011D613D6F8D508D60AD60CD60ED6F3D58D
:101A700003D605D607D609D6089507D603D6FFD5CF
:101A8000FBD5E9D502D6FED5FAD5F6D5E4D5FDD5F8
:101A9000F9D5F5D5F1D508958090B0009090B100BA
:101AA000EBD5EAD5E9D5D7D58A94D1F7EED5D3D5FC
:101AB0009A94E1F70895F894D1DF7894CADFC9DFEA
:101AC000B1E0B093B000B1E0B093B1002092B200A9
:101AD000F894E2DF7894B5E06B2E70909700C1D552
:101AE000B09197007B16C9F7B13018F0BF3F40F1B5
:101AF00007C07EDFF8944BDFB1DFB8E0B1BDA9DFEE
:101B00006A9459F7B091B200B395B093B200B33074
:101B100008F4DECF9EDFB091B100B395B093B10071
:101B2000F894B091B000BA95EEE3F0E0EB0FF21D3F
:101B3000049178940395B091B100B01708F4C6CF22
:101B400088DF87DFB091B000B395B093B000B0915B
:101B5000B000BC3008F4B7CF0DDBF89418DFB8E064
:061B6000B1BD77DFCACB26
:00000001FF
